:020000040000FA
:0400000000003F2895
:08000800A000030E8301BF00FC
:100010000A08BA0001308A00A929A601A500FF300C
:10002000A507031CA607031C3A280330A400E630EA
:100030001B200F28A401FC3EA300A409031C2628B2
:10004000FF300000A30703182128A3076400A40FB2
:10005000202808000310A30DA40DFF3E03182A2832
:1000600023083A280310A40CA30CFF3E03183228DF
:1000700023083A28831303138312640008008316AD
:1000800006309F0083120F308A0003278A010F3049
:100090008A000E278A01B700C0303707B500FF304D
:1000A0000318013EB6003508A4000B3C8A11031C5E
:1000B000832836088A11031D8328A40D8A1167201E
:1000C000A30024108A1167208A00230882000030D0
:1000D0008A002408820700348A34003490340034C3
:1000E000B0340034B9340034C6340034D23400346F
:1000F000DF340034DF340034EA340034F5340034C3
:10010000FB34013408340F308A003F3014278A0151
:100110008A0147280F308A005E3014278A01472859
:100120008512831685128312071083160710831217
:1001300087108316871083128511831685110A3064
:1001400083128A010D200714831607100A308312C8
:100150008A010D2085168316851283128A018A284A
:100160001F30C1008A11112108308A010D208A0137
:100170008A288A119E210230C1008A111121013082
:100180008A011A208A1135218A018A288A119E2122
:10019000C1018A11112101308A011A208A113521E9
:1001A0008A018A288A119E210330C1008A111121F7
:1001B00001308A011A208A1135218A018A280430E7
:1001C000C1008A11112101308A011A208A115D2192
:1001D0008A0147280530C1008A11112101308A01A6
:1001E0001A208A115D218A0147280630C1008A1130
:1001F00011218A018A281830C1008A111121013089
:100200008A010D201730C1008A1111218A018A2824
:100210000830C1008A11112108308A010D208A019D
:100220008A280130C0006400073040028A11031898
:10023000342941188515411C851101308A011A2085
:10024000871483168710013083128A011A208710C1
:1002500083168710013083128A011A200310C10C03
:10026000C00A8A11031D132908000310A10DA20D55
:100270000130C0006400113040028A1103185C296B
:1002800021188515211C851101308A011A20871437
:1002900083168710013083128A011A208710831673
:1002A0008710013083128A011A200310A20CA10CBE
:1002B000C00A8A11031D3A29080083168515831286
:1002C0000130C0006400113040028A1103188429F3
:1002D0000310A20CA10C01308A011A208714831686
:1002E0008710013083128A011A2087108316871025
:1002F000013083128A011A208519A217851DA213C5
:10030000C00A8A11031D6229851183168511031005
:100310008312220CB600210CB500FF303505A10078
:100320003F303605A2000F308A00220814270F3014
:100330008A002108142701308A0008000F308A0043
:100340000E27A2000F308A000E27A10001308A007C
:040350000800090098
:02400E00753DFE
:00000001FF
